:100800008431512CFF3FFF3F7E14843120007F084C
:10081000FB000B1D1B2C86318926843120006E0BBA
:10082000122CEE0102306E02031C182C0130EE0275
:10083000063095000B11911E2F2C0530FA00EE00AA
:1008400023001908FA007D08203E86000130870049
:100850007A0881000130FA00FD0720009112111E74
:10086000482C2100111E482C20005708580203185C
:10087000462C5808203E86000130870001082300DE
:100880009A000130FA002000D807482C21001112EC
:100890002000111B1113911891107B08FF007E108E
:1008A00009008C312C2C2100BE0146084704031D91
:1008B0005B2C002584312100490820005A02031DC9
:1008C000652C210048082000590203186F2C2100D4
:1008D00049082000DA00210048082000D900003033
:1008E0005A02513003195902031C792C5030D90097
:1008F000DA015A08DC005908DB0021003E08031920
:10090000882C3E082000AE00AF01DB002F08DC0081
:1009100020005C086002031D8F2C5B085F02031837
:10092000952C6008DC005F08DB0000305C0233308F
:1009300003195B020318BA2C0630A600A7015C0855
:10094000A1005B08A0006430A200A3018B31412309
:10095000843120002108A9002008A8008931EE2157
:100960008431200027082100E9002000260821000A
:10097000E800CF2C5B3086008701403F2000AE00AE
:10098000413FAF00AE35AF0DAE35AF0D2E08803E06
:100990002100E800023020002F3D2100E900003056
:1009A00020005C02053003195B020318DE2C2500D1
:1009B00093012000EF156F088E000800F9309B00AE
:1009C000210069082000AF00210068082000AE0067
:1009D0002F0DAF0CAE0C2F0DAF0CAE0C2E0825005A
:1009E000910003302100E8050030E9050430E835C6
:1009F000E90D890BF72C68080C3E250093000800D0
:100A0000E7302000690203181E2D21006208200033
:100A1000A0002100BE001330200069020318132D2E
:100A2000210066081A2D81302000690203181E2D4E
:100A3000210064082000A0002100BE00E730200053
:100A40006A020318080021005E082000A0002100AF
:100A5000BE00133020006A020318352D21005A0809
:100A60002000A0002100BE000800813020006A02A2
:100A70000318080021005C082000A0002100BE002F
:100A800008002000FF30A101A000A20021001D08E5
:100A900083390C389D009D149D184C2D1C08200096
:100AA000A000EB0021001D08833910389D009D1423
:100AB0009D18582D1C082000A000EC0021004608BD
:100AC0004704031D782D1D08833904389D009D14AB
:100AD0009D18682D1C082000A000EA00833021002A
:100AE0009D059D149D18722D1C082000A000E90092
:100AF00020004130A401240203189E2D21001D086E
:100B0000833908389D009D149D18842D1C082000F1
:100B1000A000A30021020318902D2308A000A1002B
:100B2000220823020318972D2308A000A2000130F9
:100B3000A000A40741302402031C7E2D2108A00040
:100B40005608A53E86008701200881000130A000DC
:100B5000D607053056060319D6010530ED01A4016C
:100B600024020318C82D2408A53E86008701010829
:100B70006D020318C12D2408A53E86000108A000BF
:100B8000ED000130A000A40705302402031CB32DA2
:100B90002208A00021004308A03E86008701200013
:100BA000200881000130A0002100C3070530430662
:100BB0000319C301FF302000A0002100BD00200068
:100BC0000530A4012402031808002408A03E860072
:100BD000870121003D0801020318F62D200024089A
:100BE000A03E86000108A0002100BD0001302000C9
:100BF000A000A4070530E22DC4302000A500A90004
:100C00002430A500A800003021004502513003190E
:100C10004402031C0E2E5030C400C50100304902AE
:100C20000E3003194802031C182E0530C800C901F4
:100C300049084502031D1E2E480844020318242EAD
:100C40004908C5004808C40000304B020C300319A5
:100C50004A02031C2E2E0130CA00CB012000AA013B
:100C600028082A020318532E2A088F31A627853117
:100C70002000A500A7002A082907A50086008701F3
:100C80000108270603194E2E2A082907A500860009
:100C90000108A600A0002A0859268531013020004D
:100CA000A500AA07302E2100CF1F0800C101C10AEC
:100CB00008002000A300A100A20123009100200051
:100CC000220823009200200020082300930095139F
:100CD000151315150B082000A100A4008B01553039
:100CE00023009600AA3096009514200024088B005B
:100CF0000330890B792E00002000121A842E033055
:100D0000890B802E00007C2E23001511200012126A
:100D10000800F90121006C0879020318C02E790837
:100D2000F6000130F635FF3E031D922E7635023E69
:100D3000523E8600013087000108F700F801F000FC
:100D40007808F10021006B08F3006A08F200D02651
:100D5000863170087104031DBC2E7908F60001303D
:100D6000F635FF3E031DB02E7635033E523E86001B
:100D7000013087008101810A0130F600F9078A2ECF
:100D80000130EA070030EB3D27306B0211300319C8
:100D90006A02031C08000130EA000030EB01080081
:100DA000700871040319F62EF501F50AF11BE12E06
:100DB0000130F035F10D890BD92E0130F400F50723
:100DC000D62E71087302031DE72E70087202031CF1
:100DD000ED2E7008F2027108F33B0130F136F00C91
:100DE000890BEE2E0130F502031DE12E7308F10090
:100DF0007208F0000800220023082000B400B501AA
:100E0000220022082000B600B701B700B60134085E
:100E10003604B90035083704BA002200250820003E
:100E2000B400BB003A08A1003908A0003B08B40098
:100E3000A200210031088A0030080A008731200012
:100E4000B500BC003C08031D282F02308C31122C49
:100E50002000BD013B083D020318502F3D35083EE0
:100E6000203E8600013087000108B4003C0886005F
:100E70008701340881000130B400BC073D35073ECE
:100E8000203E8600013087000108B4003C0886003F
:100E90008701340881000130B400BC07BD072A2F48
:100EA0000630A0018B315D23863108302000B4006C
:100EB000D700210033088A0032080A008731080071
:100EC000D2302100B4000730B500033020002102E9
:100ED000E83003192002031C852F22082007A300F5
:100EE00021080318210AA40003302402F03003195A
:100EF00023020318852F2008183EA300A5000B30FD
:100F0000E300E4012535593E080007302102D030C6
:100F100003192002031C003422082007A300210823
:100F20000318210AA40007302402E3300319230226
:100F300003180034FC302100B4000530B500200057
:100F40002008303EA300A5002535C43E0800C1346A
:100F50000834323400349C340E34143400343F34BA
:100F60000834033400342000D801FD01210011169B
:100F700023009E160800FF34FF34FF34FF34FF3493
:100F80000534FE0012001E00FE0BC22F0034640068
:100F900080010131890BC82F0034F434013401344D
:100FA000003403340800FF3FFF3FFF3FFF3FFF3F98
:10107000FF3FFF3FFF3FFF3FFF3FFF3FFF3F23009B
:101080009D1C49281D122130890B44280000230093
:101090001D16200057085802031C08006E08031D87
:1010A0000800AB22FD010800220023082000B40044
:1010B000B501220022082000B600B701B700B60132
:1010C00034083604B90035083704BA002200250870
:1010D0002000B400BB00220025352000B40022000F
:1010E000A20020003A08A1003908A0003B08B40083
:1010F000A200210031088A0030080A00883120004F
:10110000B500BC003C08031D87280230122C2000CB
:10111000BD013B083D020318AF283C08860087014B
:101120000108B4003D35043E203E860001308700B2
:10113000340881000130B400BC073C0886008701F8
:101140000108B4003D35033E203E86000130870093
:10115000340881000130B400BC07BD078928A00114
:1011600022002208033E5D2322002208053E2000C3
:10117000B400D700210033088A0032080A00883101
:101180000800073021003506031DC828D230340678
:101190000319D5288B1335088A0034080A008B17E9
:1011A000D2302100B4000730B500853141258831A7
:1011B000222288312100AE01AF014A084B04031DF1
:1011C0005B29FC302000A600A7016B08B000B1012C
:1011D000A0003108A100210045082000A300210043
:1011E00044082000A2004123883120002108A900E2
:1011F0002008A800EE21883120002708B500260825
:10120000B40001303502003003193402031C0B29ED
:10121000FF30B400B5013408B00021003A08A03E08
:101220008600013087002000300881000130B000C6
:101230002100BA0714303A060319BA01200014300D
:10124000B201B301B6013602031838293608A03EB0
:101250008600013087000108B000B101B2073108F3
:10126000B33D0130B000B60714303602031C262906
:101270001430A600A7013308A9003208A800EE2107
:10128000883120002708DA002608D9002100490803
:1012900020005A02031D502921004808200059024D
:1012A00003185E29210049082000DA0021004808BF
:1012B0002000D9005E298D319D2588310030200025
:1012C0005A0205300319590203186A290330210014
:1012D000AE00AF0121004208031D742920006118EF
:1012E000742921004F1F782903302100AE00AF017F
:1012F0005E228831003020006002053003195F0251
:101300000330031886292100AE00AF0121002E060C
:101310002F04031DA829BF2901302100AE00003091
:10132000AF01E0218831BF2902302100AE0000303A
:10133000AF01E0218831BF2902302100AE00AF01AA
:10134000200065066604031DBF29A3228831BF293A
:1013500020005E08003A0319AE29BF295D08013A52
:1013600003198C29033A03199429013A03199C297A
:10137000073A03199C29013A03199429BF2921002E
:101380002F082000E60021002E082000E50065035C
:1013900066040319D029033065066604031DD829A5
:1013A000250093012000EF156F088E00E0218831A1
:1013B0000230200065066604031D08008431532CAA
:1013C0002000671CEB29FD30A000EF056F088E00A0
:1013D0002100CF1A4F172000671008002000AB0132
:1013E000AC012608270403191D2AAD01AD0AA71B6D
:1013F000022A0130A635A70D890BFA290130AA006F
:10140000AD07F7290130AB35AC0D890B032A27084E
:101410002902031D0D2A26082802031C142A260867
:10142000A8022708A93B2B140130A736A60C890B6C
:10143000152A0130AD02031D022A2C08A7002B0833
:10144000A60008000230200065066604031D342A49
:10145000513021003D02031C342A20000530E714DE
:10146000DD000030DE0108002000D230E7106D0200
:10147000031C3F2A0130DD000030DE010800B430DB
:101480006D02031C4C2A0230DD000030DE01210019
:10149000C20120006110080095306D02031C552A1E
:1014A0000330DD000030DE0108007A306D02031CDD
:1014B00008000430DD000030DE0108002100520881
:1014C0005304031D9A2A2E3020006C0203186D2A43
:1014D0005030DF000030E00108004D306C0203188E
:1014E000762A3F30DF000030E001080080306C02D7
:1014F00003187F2A2030DF000030E0010800AE3002
:101500006C020318882A1430DF000030E001080064
:10151000D1306C020318912A0D30DF000030E00159
:101520000800210049082000E000210048082000B0
:10153000DF000800210053082000E00021005208CD
:101540002000DF000800200067180800EF146F0873
:101550008E0067140800210046084704031908009C
:1015600002307D02031C0800103022002106031DFA
:10157000C62A2608093E2000BE00003003180130AC
:10158000BF007D083E063F04031D080008307D02B1
:10159000031C0800210046082000BE00CC002200E9
:1015A000200820004C06031D0800033022002106FD
:1015B0000319E02A103021060319E02A0130122C09
:1015C000220025082000BE00BF01220023082000C1
:1015D000C000C101220022082000C200C301A000F7
:1015E0004308A100FF30A200A3014123883120005D
:1015F00040082007C4004108213DC50022002408FE
:101600002000C600C701A0004708A100FF30A200CB
:10161000A30141238831200020084407C800210885
:10162000453DC9003E084807CA003F08493DCB0078
:101630001F304B02413003194A02031808002200F0
:101640002408031D08001530250203180800200097
:10165000A001A00A7D08FE3E5D238831003A0319EF
:101660003F2B033022002106031D382B54208831E4
:10167000103022002106031D08008631FB2E0830A1
:10168000122C2000A401A501201C4A2B2208A4072B
:101690002308A53D0130A235A30D890B4B2B01304A
:1016A000A136A00C890B502B20082104031D442BCC
:1016B0002508A1002408A00008002000AD00FF308C
:1016C000B101B001AF00AE00AB012D082B022E0816
:1016D000A1002F08A2003008A3003108A4000318BD
:1016E000C82B2B08203E8600013087000108A5008A
:1016F000A601A701A801A1062608A2062708A3069D
:101700002808A4062408B1002308B0002208AF006E
:101710002108AE000830A100AC002C080319C42B2E
:101720002E1CB82B0130A100A030A200A301A401FF
:101730002E08A5002F08A6003008A7003108A80031
:101740000130A836A70CA60CA50C890BA12B2508E7
:10175000A1062608A2062708A3062808A40624082E
:10176000B1002308B0002208AF002108AE00BF2B53
:101770000130B136B00CAF0CAE0C890BB92B013077
:10178000AC022C08031D902B0130A100AB07652B88
:101790000830A436A30CA20CA10C890BC92B21087C
:1017A000A5002508AA000830AE35AF0DB00DB10D6B
:1017B000890BD42B2E08A1002F08A2003008A3000B
:1017C0003108A4000830A436A30CA20CA10C890B8C
:1017D000E32B2108A500A900200B002C2D08013EB9
:1017E000203E86000130870001082A06031D0034D0
:1017F0002D08203E86000108290603190134003413
:101800002908A1002D08203E86000130870021080C
:1018100081002A08A1002D08013E203E86002108F3
:10182000810001342000B3008030B2002200A10703
:1018300020003308B2002200A20020000330A001E3
:101840005D2305302000B200D700210033088A0054
:1018500032080A008C310800BB30840087308500D4
:10186000693086000030870006308731C1278C310F
:10187000CD30840087308500E83086000030870056
:1018800005308731C1278C31A7308400873085002F
:1018900052308600013087000C308731C1278C31EF
:1018A000FC01FD0150308400003085001930873183
:1018B000C7278C31A0308400003085004830873144
:1018C000C7278C31203084000130850032308731C9
:1018D000C7278C31A0308400013085001430873157
:1018E000C7278C317E102000752C6A3021009900AA
:1018F000FF308C00E1308E0008302000CF00EF0078
:101900008E00603021009E001D141D0883390838A8
:101910009D002500161522001E11013021009500A2
:1019200024000C148C140C118C110C168C120E103B
:101930004F258C3121001708C1391638970017142C
:101940006C278C3120000030D001D10151020530CC
:10195000031950020318C22CFF30CF005008A53ED7
:10196000860087014F0881005008A03E86000130A4
:101970008101D0070030D13D5102053003195002DA
:10198000031CAC2C210046084704031D192D200020
:101990000930D001D1015102C4300319500203189B
:1019A000112D21001D0883390C389D009D149D18B0
:1019B000D72C1C082000CF00EB0032306B0203183C
:1019C000EF2C21003608031DEF2C01302000CF0042
:1019D0002100B70773278C312100B601B60A210018
:1019E00036080319002D653020006B02031C002D02
:1019F0000130CF002100B7076C278C312100B601E0
:101A00006400BE300032890B022D01302000D00767
:101A10000030D13D09305102C43003195002031C7B
:101A2000D12C0A3021003702031C192D0130C600C9
:101A3000C70173278C31B3302100B2000730B300E7
:101A40006030B0000730B100D230B4000730B500CC
:101A50004608470403192E2DB5278C318B170B1719
:101A6000210091148B16053020009C0021004508B0
:101A70002000DA00210044082000D900FD30DD01FB
:101A8000DE016710CF00EF056F088E000130E50022
:101A90000030E6002100CF13C4278C314C2DC43018
:101AA0002000AB00AD002530AE012E0203186B2DD7
:101AB0002E08A6278C312000AB002E082D07AC0085
:101AC000860087012B0881000130AB00AE0725306E
:101AD0002E02031C582D2100580F0800590F080032
:101AE0002030C4000530C501C601C701C80001305F
:101AF000C901CA00CB01CC01CD01CE000630CF0117
:101B0000D001D101D201D301D8000A30D901DA00C5
:101B10001030DB01DC001930DD01DE002030DF0198
:101B2000E0003030E101E2003F30E301E4005030FA
:101B3000E501E600E7018531FC2D323020006B0223
:101B4000003003185C2E53020B3003195202031CA1
:101B5000B62D2100CE1CB62D033020005D065E049C
:101B6000031DB62D2100C201C20A080021004E1C2F
:101B700008000030200053021F3003195202031CDA
:101B8000562E1F3052065304031DED2D2100B801BF
:101B9000B90120001430D50155020318ED2D6C2732
:101BA0008C310D302000A600FB30890BD52DA60B03
:101BB000D52D003273278C310D302000A600FB306C
:101BC000890BE02DA60BE02D003201302000A6008D
:101BD000D50714305502031CCF2D0630A000A101FB
:101BE0005308A3005208A2007A278C310430200049
:101BF00020062104031D462E21004A084B04031928
:101C00000D2E00304B020B3003194A0203180D2E23
:101C10004A082000A6002100B8070B304A064B04F2
:101C2000031D1F2E0930390203181F2E3935D83EE7
:101C30008600870101082000A6002100B8003808AE
:101C40002000A600A7012100490820002702031D4B
:101C50002D2E21004808200026020318382E2100CE
:101C600049082000DA00210048082000D900402E51
:101C7000210038082000A600A701D9002708DA00B3
:101C80000130A6002100B9076C278C3106302000F6
:101C9000A000A1015308A3005208A2007A278C31AA
:101CA000200020082104031D562E73270130200038
:101CB000D2070030D33D080053021F3003195202EF
:101CC000031C992E1430D50155020318852E6C275C
:101CD0008C310D302000A600FB30890B6D2EA60B39
:101CE0006D2E003273278C310D302000A600FB30A2
:101CF000890B782EA60B782E003201302000A6002A
:101D0000D50714305502031C672E21004C084D04E2
:101D10000319962E20005A082100C50020005908FA
:101D20002100C400FC30B4000530B5002000D20111
:101D3000D301D201D3010800210041080319640036
:101D400021004F1BB62ED62E6C278C31CB2E73273D
:101D50008C31CB2E6C278C31CB2E73278C31CB2E34
:101D60006C278C31CB2E73278C31CB2E200054085E
:101D7000013A0319A42E053A0319A72E033A0319B1
:101D8000AA2E0D3A0319AD2E073A0319B02E1D3AAB
:101D90000319B32ECB2E333020005402031CD22E55
:101DA000D40108000130A100D40708002000E71882
:101DB000F82E242F6C278C31192F73278C31192F73
:101DC0006C278C31192F73278C31192F6C278C318C
:101DD000192F73278C31192F6C278C31192F7327EA
:101DE0008C31192F6C278C31192F73278C31192FB7
:101DF00020005408013A0319DA2E053A0319DD2EA2
:101E0000033A0319E02E0D3A0319E32E073A03199A
:101E1000E62E1D3A0319E92E043A0319EC2E033A73
:101E20000319EF2E0C3A0319F22E053A0319F52E79
:101E3000192F473020005402031C202FD401080022
:101E40000130A100D407080052085304031D080004
:101E50005D035E04031D362F7C08031D322F6C27A3
:101E60008C31362F7C0B362F73278C3102302000BB
:101E70005D065E04031D522F7C08031D422F6C2754
:101E80008C31522F7C0B452F502F05307C06031DC3
:101E90004C2F6C278C31522F06307C06031D522F9D
:101EA00073278C31033020005D065E04031D632F11
:101EB0007C08031D5E2F6C278C31632F0A307C0653
:101EC000031D632F732701302000A100FC0715308C
:101ED0007C020318FC01080014302000A000EF046D
:101EE0006F088E000800EB302000A000EF056F089F
:101EF0008E0008002000200821040319A12FA5014D
:101F0000A50AA11B8C2F0130A035A10D890B842FB0
:101F10000130A400A507812F21082302031D922F61
:101F200020082202031C982F2008A2022108A33BAC
:101F30000130A136A00C890B992F0130A502031D99
:101F40008C2F2308A1002208A00008002000A20076
:101F5000A000A1012300910020002108230092008D
:101F60009513151315141308080022009D171D154D
:101F700023001E159C0119309B001E129D171D1673
:101F80008C102100911608002000CE0121006C0861
:101F900020004E02031808004E08CD000130CD3558
:101FA000FF3E031DCF2F4D35033E523E86000130CC
:101FB000870001080319FC2F4E08CD000130CD35F4
:101FC000FF3E031DDF2F4D35523E86000130870056
:101FD000413F8A00403F0A008F3120004E08CD006B
:101FE0000130CD35FF3E031DF12F4D35033E523EEE
:101FF00086000130870081010130CD00CE07C62F59
:020000040001F9
:04000E00BCF9FFDE5C
:00000001FF
